:107800005CC000008FC0000073C0000071C00000A9
:107810006FC000006DC000006BC0000069C00000B8
:1078200067C0000065C0000063C0000061C00000C8
:107830005FC000005DC000005BC0000059C00000D8
:1078400057C0000055C0000053C0000051C00000E8
:107850004FC000004DC000004BC0000049C00000F8
:1078600047C0000045C00000040309041C03770062
:10787000770077002E0066006900730063006800DF
:107880006C002E00640065000E035500530042009A
:1078900061007300700012011001FF000008C016A3
:1078A000DC05020101020001090212000101008051
:1078B0003209040000000000000011241FBECFEFB9
:1078C000D8E0DEBFCDBF11E0A0E0B1E0E4ECFFE71F
:1078D00002C005900D92A630B107D9F711E0A6E0DD
:1078E000B1E001C01D92AD33B107E1F73CD168C3EF
:1078F00087CFA82FB92F80E090E041E050EA609553
:1079000030E009C02D9182279795879510F0842744
:107910009527305EC8F36F5FA8F30895EADF8D9373
:107920009D930895CF93CFB7CF93DF93C3954C9B8F
:10793000E9F74C9B0BC04C9B09C04C9B07C04C9B70
:1079400005C04C9B03C04C9B01C089C06F93C09184
:107950002001DD27C95DDE4F2F9365E54C9B03C0F9
:107960002F916F91E6CF0F931F934F9320E040E14B
:107970005F9309B1047104FB27F93F9350E03BE0AA
:1079800039C0147140642F77012F5F5F1EC04068BB
:1079900019B114712F7752501FC0406409B12F776D
:1079A0000471D1F15F5F00C023C0406219B12F772D
:1079B000147191F15F5F00C025C004711027515010
:1079C00012F45D5F0000115027952C3F19B1C8F6E5
:1079D00014710127015027952C3FC8F6422749937F
:1079E00009B1047110274F73115027952C3FA8F649
:1079F0004695469519B1147179F0012701502795E4
:107A00002C3F98F66B5A60F3315009B1B0F600C0C4
:107A100011E01CBB002717C03B503195C31BD04061
:107A200011E01CBB0881033CF9F00B34E9F0209114
:107A30001E011981110F1213EDCF093651F10D32CC
:107A400011F0013E39F7009325013F915F914F916D
:107A50001F910F912F916F91CCB3C0FD67CFDF9134
:107A6000CF91CFBFCF91189520912501222369F3A3
:107A700010912301112339F534303AF13093230169
:107A800020931F01109120013BE0311B3093200116
:107A90001CC0009123010130B4F40AE530910001CB
:107AA00034FD14C000930001C3E1D1E013C00527E9
:107AB00010E000C000000BB91AC0052710E0221F1B
:107AC0001DC010E021C04AE502C032ED432FC4E1E1
:107AD000D0E032E01AB114615C9A0BB11AB954E1EA
:107AE00020E865E320FF05270BB9279517951C3F74
:107AF000F0F66695B8F7B1F720FF05270BB9279583
:107B000017951C3FD0F62795179517FF05270000FE
:107B10001C3F0BB9B0F629913A9519F70B7E1091DD
:107B20002401110FC651D0400BB911F010931E0162
:107B300011E01CBB00611AB11B7E402F4B7E54E04C
:107B40005A95F1F70BB91AB94BB97FCF1BB8F89416
:107B50001DBA1092690081E085BF15BEE091110148
:107B6000F0911201099588E10FB6F89480936000B6
:107B7000109260000FBE5F9A04B601FE0AC214BEE6
:107B800081E085BF82E085BF4F9903C28091690083
:107B9000826080936900E89A549A20E005C0A89515
:107BA00080EA9FE00197F1F72150C9F75498789443
:107BB000CC24DD2490912301935097FD61C18091E5
:107BC00020010CE010E0081B1109095D1E4F809197
:107BD0001F018D3209F0DDC0983009F04FC183ECF0
:107BE000809313018AE58093000110920A01D80165
:107BF0003C91832F807611962C911197882309F45C
:107C000051C086E091E090932201809321012330BE
:107C1000F9F413969C91139714968C9114971296DD
:107C20002C91203339F48370E82FF0E0EE5FFE4FA3
:107C300080810AC0203A11F4ADD106C0203C19F46D
:107C4000F8016581AFD180E08093090194E093C091
:107C5000253011F491E08FC0822F84508630D8F403
:107C6000D80112968D919C91139790930D0180935A
:107C70000C012930A9F016969C91169790930E014D
:107C800015968C91827080930F012093100137FD1F
:107C90006DC02FEF6CC0223019F481E080930B018E
:107CA00090E069C0F801828110921C01222331F416
:107CB00010921D012CE131E092E053C0253019F4FF
:107CC000809324014BC02630C9F5D80113968C91BE
:107CD000813019F486E998E704C0823041F488EADB
:107CE00098E7909322018093210192E123C0833091
:107CF00001F5F8018281882341F488E698E79093A2
:107D000022018093210194E015C0813041F48CE67A
:107D100098E790932201809321019CE10BC082306F
:107D200041F488E898E790932201809321019EE036
:107D300001C090E080E480930A011DC0283019F44E
:107D400026E231E009C0293019F48093260106C0EB
:107D50002A3021F42CE131E091E003C02CE131E044
:107D600090E0309322012093210105C0292F80E863
:107D700080930A010BC0D80117968C91179788231E
:107D800021F416962C91291708F0292F2093010130
:107D900075C080910A0187FF71C080910E01F92E94
:107DA000891708F4F82E8F1980930E01EE2488238A
:107DB00011F4EE24E39480911001873010F0E80173
:107DC00014C050910F01E0910C01F0910D0140E0C1
:107DD0004AC080910C0190910D01019690930D0184
:107DE00080930C0101976991DDD0FE01E01BEF1536
:107DF00080F340C0CF018F779070892B49F4F894BD
:107E000083E080935700E895789407B600FCFDCF97
:107E10004E5FF894D8018D919D918D0121E00C0168
:107E200020935700E895112478949F012E5F3F4FCF
:107E3000C9018F779070892B31F0EE2099F04F15A2
:107E400088F0552379F0F89485E080935700E89501
:107E5000789407B600FCFDCFF89481E18093570039
:107E6000E8957894F9014F1508F4C4CFF0930D010B
:107E7000E0930C01EE2011F0109201011092230109
:107E80008091000184FF71C0809101018F3F09F44E
:107E90006CC0182F893008F018E0811B8093010115
:107EA0008091130198E8892780931301112309F425
:107EB0004AC080910A0187FF2AC080910E01811774
:107EC00008F4182F811B80930E0100911001C4E16A
:107ED000D1E015C0E0910C01F0910D01073018F0D0
:107EE000CF0158D001C084918883219680910C01E4
:107EF00090910D01019690930D0180930C01812FBB
:107F000090E08C5E9E4FC817D90721F71AC0E09108
:107F10002101F091220186FF09C0912FA4E1B1E077
:107F200084918D9331969150D9F707C0912FA4E198
:107F3000B1E081918D939150E1F7F0932201E093AC
:107F40002101193060F484E191E0612FE7DC612FB9
:107F50006C5F6C3041F08FEF8093010104C08FEFB4
:107F6000809301016EE16093000194E189B1847115
:107F700031F49150D9F71092240110921E01809192
:107F80000B01882321F0CA9411F4DA9411F04F9B6D
:107F900011CEDCDDF999FECF92BD81BDF89A99270B
:107FA00080B50895262FF999FECF1FBA92BD81BDE5
:107FB00020BD0FB6F894FA9AF99A0FBE019608956B
:047FC000F894FFCF63
:067FC4005AFF1E950F009C
:040000030000780081
:00000001FF
